:1000000012C0189518951895189518951895189563
:100010001895189518951895189518951895189578
:100020001895189518958FE58DBFC0E4E0E34E2E26
:1000300084E08EBFD4E0F4E05F2EEEEFF3E0A0E6C4
:10004000B0E088278D933197E9F789E189B980E09D
:1000500080BD88E18AB966248EE181BD86E181BDDB
:10006000A098A198A298A398A498A5988A9A8B9AE8
:100070008C9A8D9A8E9A8F9A929893989498959834
:100080009698979880E08093BC0080E08093C100B0
:100090008BE18093BA00AAEBB0E08C91A5EBB0E0C5
:1000A0008D9388278C93A5EBB0E0B5D4EEEFF2E109
:1000B000ECD65FD2E0E0F0E0A2ECB0E001D9E1E004
:1000C000F0E0A3ECB0E0FCD8E2E0F0E0A4ECB0E0BB
:1000D000F7D80091C2000F3F09F00BC00091C30098
:1000E0000F3F09F006C00091C4000F3F09F001C0A6
:1000F00014D4E2E0F0E0B3D4FDD33BD2EFD10091D1
:10010000C200003009F078C081B5886081BDA19837
:10011000A09890E2A0E6B0E0983018F4392F992723
:1001200002C038E098509999FECF88949899089425
:100130008795999BFECF3A95B1F78D93992361F7F7
:10014000A89501D1CBD10091C100013009F00CC0BC
:10015000EAEFF2E126D7EDEBF0E09CD6B4D4EDE087
:10016000F0E0ADEBB0E080D80091BC00003009F0C9
:100170002FC0AAEBB0E08C916ED4E2E0F3E162D440
:10018000A0EAB0E059D4A8E1B4E0A8E1B4E0EDEB16
:10019000F0E0552743E0EDD44DD4EAD20091C10000
:1001A000013009F014C0AAEBB0E08C9154D4EAE01D
:1001B000F3E148D4E2E1F3E145D4AAEBB0E08C915D
:1001C0004AD4E2E2F3E13ED4EAE2F3E13BD414C0E4
:1001D000AAEBB0E08C913FD4E2E0F3E133D4A4E6A3
:1001E000B0E02AD4AAEBB0E08C9135D4E2E2F3E19E
:1001F00029D4EAE2F3E126D40091C300003009F0EB
:100200004EC081B5886081BDA398A29890E2A0E617
:10021000B0E0983018F4392F992702C038E0985090
:100220009B99FECF88949A99089487959B9BFECFC3
:100230003A95B1F78D93992361F7A89584D04ED163
:100240000091BC00003009F016C0AAEBB0E08C9120
:1002500002D4ECE2F3E1F6D3A0EAB0E0EDD3A8E1FA
:10026000B4E0A8E1B4E0EDEBF0E0552743E081D441
:10027000E1D37ED214C0AAEBB0E08C91ECD3ECE2D7
:10028000F3E1E0D3A4E6B0E0D7D3AAEBB0E08C91E1
:10029000E2D3E2E2F3E1D6D3EAE2F3E1D3D3009191
:1002A000C400003009F04EC081B5886081BDA598BA
:1002B000A49890E2A0E6B0E0983018F4392F99277E
:1002C00002C038E098509D99FECF88949C9908947C
:1002D00087959D9BFECF3A95B1F78D93992361F752
:1002E000A89531D0FBD00091BC00003009F016C0B9
:1002F000AAEBB0E08C91AFD3E4E3F3E1A3D3A0EA9F
:10030000B0E09AD3A8E1B4E0A8E1B4E0EDEBF0E00E
:10031000552743E02ED48ED32BD214C0AAEBB0E0E5
:100320008C9199D3E4E3F3E18DD3A4E6B0E084D3D8
:10033000AAEBB0E08C918FD3E2E2F3E183D3EAE25F
:10034000F3E180D3DCCEA4E6B0E0E0E6F0E06BD7EA
:100350008CE1E4E6F0E004E00A93A5E8B0E08AD797
:1003600088E1E4E6F0E004E00A93AAE8B0E082D78E
:1003700084E1E4E6F0E004E00A93AFE8B0E07AD785
:1003800080E1E4E6F0E004E00A93A4E9B0E072D78B
:100390008CE0E4E6F0E004E00A93A9E9B0E06AD773
:1003A000A5E8B0E04FD7A4EAB0E00D931C93AAE80B
:1003B000B0E048D7A6EAB0E00D931C93AFE8B0E0F8
:1003C00041D7A8EAB0E00D931C93A4E9B0E03AD776
:1003D000AAEAB0E00D931C93A9E9B0E033D7ACEAE8
:1003E000B0E00D931C9387E0E4E6F0E001E00A93AF
:1003F000AEE9B0E03FD7AEE9B0E0ECE3F3E16AD7B5
:1004000009F006C0A0EAB0E0EEE3F3E13ED505C096
:10041000A0EAB0E0E0E4F3E138D585E0E4E6F0E01E
:1004200001E00A93A2EAB0E025D7A2EAB0E0E2E454
:10043000F3E150D709F02CC0AEEAB0E0ECEAF0E00E
:100440009DD6AEEAB0E0E7D2EAEAF0E097D6AEEAAF
:10045000B0E0E1D2E8EAF0E091D6AEEAB0E0DBD27B
:10046000E4E4F3E112D5AEEAB0E0D5D2E6EAF0E09A
:1004700085D6AEEAB0E0CFD2E4EAF0E07FD6AEEACD
:10048000B0E098D5EDE0F0E0ADEBB0E0EDD625C002
:10049000AEEAB0E0EAEAF0E071D6AEEAB0E0BBD294
:1004A000E4E4F3E1F2D4AEEAB0E0B5D2E8EAF0E099
:1004B00065D6AEEAB0E0AFD2E6EAF0E05FD6AEEAEB
:1004C000B0E0A9D2E4EAF0E059D6AEEAB0E072D5E5
:1004D000EDE0F0E0ADEBB0E0C7D60895A3D2ABEB12
:1004E000B0E08C930091BB00003010F009F001C027
:1004F0003FC082E6482F0091BB00041709F003C0FB
:1005000081E08093BC0083E6482F0091BB00041774
:1005100009F001C089D184E6482F0091BB0004177F
:1005200009F006C080E08093BC0080E08093C100A9
:1005300085E6482F0091BB00041709F001C0EDD1FA
:1005400086E6482F0091BB00041709F001C041D195
:1005500082E7482F0091BB00041709F003C081E037
:100560008093C1000091BB000B3109F001C001D0A4
:100570000895A5EBB0E060D2AAEBB0E08C916BD20D
:10058000E6E4F3E15FD2AAEBB0E08C9164D2ECE454
:10059000F3E158D2A5EBB0E04FD2AAEBB0E08C91DA
:1005A0005AD2E2E5F3E14ED2EAE5F3E14BD250D282
:1005B000AAEBB0E08C914FD2ECE7F3E143D2E4E850
:1005C000F3E140D245D2AAEBB0E08C9144D2ECE901
:1005D000F3E138D2E2EAF3E135D2AAEBB0E08C9154
:1005E0003AD2ECEAF3E12ED2E2EBF3E12BD2AAEB22
:1005F000B0E08C9130D2ECEBF3E124D2E2ECF3E109
:1006000021D2AAEBB0E08C9126D2E2E2F3E11AD239
:10061000EAE2F3E117D2AAEBB0E08C911CD2ECEC49
:10062000F3E110D2AAEBB0E08C9115D2E0EDF3E14A
:1006300009D2E8EDF3E106D2AAEBB0E08C910BD23F
:10064000EAEFF3E1FFD1E2E0F4E1FCD1AAEBB0E0A4
:100650008C9101D2E4E2F4E1F5D1ECE2F4E1F2D1E3
:10066000AAEBB0E08C91F7D1EEE4F4E1EBD1E6E552
:10067000F4E1E8D1AAEBB0E08C91EDD1E8E7F4E148
:10068000E1D1E0E8F4E1DED1AAEBB0E08C91E3D176
:10069000E2EAF4E1D7D1EAEAF4E1D4D1AAEBB0E09E
:1006A0008C91D9D1ECECF4E1CDD1E4EDF4E1CAD1F7
:1006B000AAEBB0E08C91CFD1E6EFF4E1C3D1EEEF3D
:1006C000F4E1C0D1AAEBB0E08C91C5D1E0E2F5E154
:1006D000B9D1E8E2F5E1B6D10091C2000F3F09F0CF
:1006E00014C0AAEBB0E08C91B6D1E2E0F3E1AAD15C
:1006F000EAE4F5E1A7D1AAEBB0E08C91ACD1E2E25B
:10070000F3E1A0D1EAE2F3E19DD10091C3000F3FF4
:1007100009F014C0AAEBB0E08C919DD1ECE2F3E1BA
:1007200091D1EAE4F5E18ED1AAEBB0E08C9193D1BE
:10073000E2E2F3E187D1EAE2F3E184D10091C4007F
:100740000F3F09F014C0AAEBB0E08C9184D1E4E330
:10075000F3E178D1EAE4F5E175D1AAEBB0E08C9150
:100760007AD1E2E2F3E16ED1EAE2F3E16BD10895EE
:10077000A2EAB0E0E2E4F3E1ADD509F015C0EEE5A0
:10078000F5E160D1AAEBB0E08C9165D1ECECF3E13E
:1007900059D1AAEBB0E08C915ED1E2E2F3E152D103
:1007A000EAE2F3E14FD114C0E2E6F5E14BD1AAEB66
:1007B000B0E08C9150D1ECECF3E144D1AAEBB0E085
:1007C0008C9149D1E2E2F3E13DD1EAE2F3E13AD1A1
:1007D0000895929A88E290E051D1929888EC90E046
:1007E0004DD1939A88E290E049D19398A895959A33
:1007F00088E290E043D1959888EC90E03FD1949ABC
:1008000088E290E03BD19498A895979A88E290E08E
:1008100035D1979888EC90E031D1969A88E290E0B3
:100820002DD19698A8950895AAEBB0E08C9113D19C
:10083000E2E2F3E107D1E8E6F5E104D1AAEBB0E0AA
:100840008C9109D1ECECF3E1FDD0ECD0ABEBB0E056
:100850008C93A8950091BB00003010F009F001C006
:100860002FC08AE7482F0091BB00041709F006C08B
:10087000939A8CE291E002D19398A89589E7482F4A
:100880000091BB00041709F006C0949A8CE291E035
:10089000F5D09498A89588E7482F0091BB000417DD
:1008A00009F006C0969A8CE291E0E8D09698A89557
:1008B00081E6482F0091BB00041709F001C01AD04F
:1008C0000091BB00003010F009F001C0BECFAAEBD0
:1008D000B0E08C91C0D0E2E2F3E1B4D0EAE2F3E11F
:1008E000B1D0AAEBB0E08C91B6D0ECECF3E1AAD099
:1008F000A8950895939A8CE291E0C0D09398A8951A
:10090000949A8CE291E0BAD09498A895969A8CE249
:1009100091E0B4D09698A8950895AAEBB0E08C9198
:100920009AD0E2E2F3E18ED0EAE2F3E18BD0AAEBD7
:10093000B0E08C9190D0ECECF3E184D0ECE8F5E100
:1009400081D070D0ABEBB0E08C930091BB00003055
:1009500010F009F001C055C088E7482F0091BB0096
:10096000041709F00BC080E08093C200E0E0F0E0E3
:10097000A0E1BB2780E08C937BE791D489E7482FE7
:100980000091BB00041709F00BC080E08093C30006
:10099000E1E0F0E0A0E1BB2780E08C937BE77FD42F
:1009A0008AE7482F0091BB00041709F00BC080E0D4
:1009B0008093C400E2E0F0E0A0E1BB2780E08C93EC
:1009C0007BE76DD48CE6482F0091BB00041709F03B
:1009D00018C0E0E0F0E0A0E1BB278FEF8C937BE74D
:1009E0005ED4E1E0F0E0A0E1BB278FEF8C937BE7E2
:1009F00056D4E2E0F0E0A0E1BB278FEF8C937BE7D9
:100A00004ED4A8950091BB000D3009F09ACFB1DD0E
:100A10000895F894FFCF8F938D918823E9F711976C
:100A20008F91089588275F9B089500C05F9BFECF3C
:100A30008CB10895A8E1B4E08D91882311F00BD01A
:100A4000FBCF0895AAD2802D11F005D0FBCF0895D9
:100A50008DE001D08AE05D9BFECF8CB9089588EED1
:100A600093E00CD03197D9F708953197F1F70895B5
:100A7000689462F80895E89462F80895EF93FF93FC
:100A8000EE27E82BE92B31F0E0EAFFE03197F1F7B0
:100A90000197D1F7FF91EF9108958F939F93D2160D
:100AA000E306F4060FB680E890E8802795270FBE8E
:100AB00089070FB6892B87FD02C091E009260FBE7A
:100AC0009F918F91089543D0A9F0503899F016273F
:100AD000050F1BF40AF038C23EC203951BD0FF205D
:100AE0002AF0BB0CDD1CEE1CFF1C02C003951BF0A2
:100AF00003D0DAC130C228C2B7FE089590E8B91613
:100B000011F4D0FE08959FEFD91AE90AF90A09F401
:100B100003950895FF92EF928D2DFF24EE24DD249E
:100B2000BB2493E0849F1001829FB00CD11CE21C77
:100B3000F31C839FD00CE11C2224F21C9A9531F007
:100B4000BD2CDE2CEF2CFF248F91ECCF0895652F68
:100B500090E8440F551F5927990F47956078102F3B
:100B600090E8FF0C001F0927990FF79410780038C0
:100B7000089590D1F4DF17FF03C08DE28D93112704
:100B8000003819F4EEE2FEE080C10F3741F4FF2097
:100B900019F4E4E2FEE0F8CFE0E2FEE0F5CF4A939C
:100BA0004A934A935A93BA93AA93BB270F5FCAF406
:100BB000BB27802F0A9578D18D3E70F4EEE7FEE0DA
:100BC000A3E0EFD16ADFBB1FB0FF04C07097E9D18B
:100BD0007ADF3C96AA95A9F7EAE7FEE0E2D173DF57
:100BE0001DC0093028F1033148F10A3130F418E012
:100BF0008BE192E9E2E3FEE028C00A9555D1E2E7F5
:100C0000FEE0BFEFA3E0CDD148DFBB1FB0FD04C0C5
:100C10003896C7D158DF3C97AA95A9F7B095BB0F76
:100C20009EDF039513E08AEF99E0F816090740F478
:100C300013E08BE094E0E6E4FEE007C016E001C0BC
:100C4000B39583E194E2EAE3FEE06A81BF3F19F4E1
:100C5000BB2711276260BD836A831C83A881B98189
:100C600060E36D93A883B9836D93081B0195AA2453
:100C7000BB246A816A7F002339F0F694E794D79405
:100C8000B794A7940A95F7CF19E000278AD1CC240E
:100C90008FEF74E0AC14B206D306E406F50630F02C
:100CA000AC18B20AD30AE40AF50A21F1881F7A9532
:100CB00031F05695479537952795C794EBCF80959A
:100CC00022D041F0969510F7FE2CED2CDB2CBA2C9F
:100CD000AA24DCCF25D05D813C812B8170D0277088
:100CE00021F02BD06CD0E8F301C03CD04CD078D0B0
:100CF000269608958894881F7A95E9F7809503D001
:100D000049F38827FCCF806360FD06C0803311F073
:100D1000616002C0039561FD8D9360FD1A95089591
:100D200099278E919C9385338E9108F083958A3311
:100D300008F080E38C93C0F70895732F720F61FF62
:100D4000701B0AD01296785019F050F38E9380E3FE
:100D50008E937150EAF70895A881B981A70F88276B
:100D6000B81F089579E061FD700FF6DF48E0431B7E
:100D7000400F8AF381F399274A9569F38E91803366
:100D800051F79C93F9CF732F61FF701B7395A88166
:100D9000B981EA2FFB2F11978191803361FF09F010
:100DA0008D937A9511F48EE28D9381918823C1F70A
:100DB000772311F480E38D9388278C93089588948A
:100DC00062FD0895002359F4A881B9818C91803384
:100DD00031F0552321F05395335064600894089501
:100DE0005523E9F085E48D931AF48DE28D935195A6
:100DF000652F660F560F5A3010F060E503D068E09B
:100E000001D0DACF8FEF74E0561708F0561B881F19
:100E10007A9511F06695F8CF809580638D9308954B
:100E20004E414E00496E66696E6974790000302E3D
:100E3000300000404B4C0020A107000050C30000D0
:100E400088130000F40100000032000000050000DB
:100E50008000CCCCCC0C14AE47019CC42000DC46F6
:100E60000300E353000063080000D70000001500F2
:100E700000001CC25367A5D468530024744915BEF2
:100E80009A17CCBC8C2BBD37863587D00D920020AD
:100E9000E1F70895D190E190F190019108952191A9
:100EA0003191419151910895FF0C90E89027110FD5
:100EB0009795F794092F0895502F2D2D3E2D4F2DE6
:100EC000612F08952DEC3CEC4CEC5DE366270FC0E0
:100ED000E1DFF2DFDD24EE2490E8F92E0FE307C016
:100EE000DEDF05C02227332740E251E46627552381
:100EF00051F1002381F12BDE71F116270058505873
:100F00000894050B18F407FD03C025C007FD23C096
:100F1000469537952795F694E794D79422D0FF20ED
:100F20002AF0DD0CEE1CFF1C015073F09D2D9695F0
:100F300048F0DD203AF4EE202AF491E0D90E99270A
:100F4000E91EF91EB1CF07C09FE7092FF92A9FEFCD
:100F5000D92EE92E0895DD24EE24FF240027112741
:100F600008959F929924AA24BB2488E1D216E3060F
:100F7000F40628F0D21AE30AF40A089401C088940F
:100F8000991CAA1CBB1CDD0CEE1CFF1C8A9571F77A
:100F9000D92CEA2CFB2C9F900895C89531960020FF
:100FA0000895FBDF202DF9DF302DF7DF402DF5DF31
:100FB000502D089560DDE89488278A938A93CBDFCB
:100FC00011278D918032E9F31197BAD090F08D32CC
:100FD00029F4109511968C91B3D058F08E3229F4E3
:100FE00011968C91ADD008F445C0229641DD81E088
:100FF00008958C91A5D0D8F547D01196D0F70395D8
:101000008D919ED0E0F38E3229F48C9199D010F41A
:101010001196FBCF853419F0853609F055C011962D
:101020008C918ED060F08D3219F08B3221F0DDCFB3
:1010300008800094088211968C9182D0B0F680537B
:10104000898311968C917CD058F49981990F990FCE
:101050000980900D990F8053890F8983873228F674
:101060008981988199230AF48195080F2DC08E32C9
:1010700089F611968C9164D068F606D018F0119616
:101080000A95F8CF1196C1CF4F2D3E2D2D2DDD0C99
:10109000EE1CFF1CA8F0DD0CEE1CFF1C88F0D20E2D
:1010A000E31EF41E68F0DD0CEE1CFF1C48F08053BC
:1010B00009F06894D80E8827E81EF81E08F00895F5
:1010C000F42EE32ED22E089534D019F116F50983AB
:1010D00008E921D00695882787959F2D9F77980F3F
:1010E000F92E0150000F110F07958981882379F09F
:1010F0001AF48195898306C0E5DE89818A95898302
:10110000D9F705C0EFDE89818A958983D9F72296C0
:10111000089521DFFCCF0DD041F0FF2032F00A9579
:1011200031F0DD0CEE1CFF1CD2F788940895089472
:10113000089500240D280E280F28002A0020089565
:10114000803320F08A3310F4089408958894089529
:10115000000F111F221F331F089500951095209531
:1011600030950F5F1F4F2F4F3F4F08950191108112
:101170000EC001911191219130810BC0019110811C
:1011800017FF05C03FEF2FEF04C000811127222772
:10119000332737FF03C0E1DF8DE28D93CF93DF93D9
:1011A000CF92DF92EF92AA24BB24CC24DD24EE243C
:1011B00040E2CAE0DD2755E093E38881890F87FD8F
:1011C0009F7083FD907F891B89935A95A9F7C0DF93
:1011D000AA1CBB1CCC1CDD1CEE1C4A9551F7E894E4
:1011E000EFE0FF2782910ED0EB30E0F71EF068941D
:1011F0008A2D0CD088278D93EF90DF90CF90DF91D0
:10120000CF910895982F829501D0892F8F70805D9E
:1012100026F0803309F4089568948D93089541E091
:1012200003C042E001C044E0E40F8827F81F829128
:1012300038E098E1880F991F9D933A95D1F74A9528
:10124000B1F70FC000271127222733278D9188235C
:1012500039F08053000F111F221F331F080FF6CFE4
:10126000089588278D93089594E081918D939A95A0
:10127000E1F7089509919191992351F08A95D9F751
:10128000319781918D930A9519F08823D1F70895AC
:10129000E8CFE199FECFEEBBFFBB3196089591E018
:1012A00001C092E07B3751F47FB7F894F2DF8D9163
:1012B0008DBBE29AE19A9A95C9F77FBF7727089587
:1012C00091E001C092E0E5DFE09A8DB38D939A95AD
:1012D000D1F70895689401C0E894AF93BF938D91BE
:1012E00016F0919102C059DE902D891718F011F473
:1012F0008823A9F7BF91AF910895000000405B32A9
:101300004A005B353B31344800005B353B323548A1
:101310000000202D2044757263686D6573736572DB
:1013200000005B31313B344800003E005B373B310D
:10133000344800005B393B313448000030002B005A
:101340002D0031002E005B34306D00005B33376DB3
:1013500000005B313B32304800004D6573737363AE
:10136000686965626572204175736C6573652053A9
:10137000797374656D2056312E3000005B323B323C
:1013800035480000A92048616E7320426F726E6775
:101390007261656265722032303038005B353B34F3
:1013A0004800582D4163687365203A005B373B3431
:1013B0004800592D4163687365203A005B393B341E
:1013C00048005A2D4163687365203A005B4B00006A
:1013D0005B31333B32480000C9CDCDCDCDCDCDCD35
:1013E000CDCDCDCDCDCDCDCDCDCDCDCDCDCDCDCD2D
:1013F000CDCDCDCDCDCDCDCDBB005B31343B324855
:101400000000BA20622020203D2062696E61657272
:1014100020202020202020202020202020202020CC
:101420002020BA005B31353B32480000BA206320EF
:1014300020203D20636C6561722020202020202028
:10144000202020202020202020202020BA005B31D6
:10145000363B32480000BA20642020203D206465DD
:101460007A696D616C2020202020202020202020FF
:10147000202020202020BA005B31373B324800007A
:10148000BA20652020203D2065696E72696368740A
:10149000656E2020202020202020202020202020B9
:1014A000BA005B31383B32480000BA206620202069
:1014B0003D206661737420726561642065696E2FDA
:1014C00061757320202020202020BA005B31393B39
:1014D00032480000BA20722020203D2044757263FB
:1014E000686D65737365722F52616469757320202E
:1014F00020202020BA005B32303B32480000BA2066
:10150000455343203D2042696C6473636869726D82
:10151000206E657520617566626175656E20BA0022
:101520005B32313B32480000C8CDCDCDCDCDCDCDE5
:10153000CDCDCDCDCDCDCDCDCDCDCDCDCDCDCDCDDB
:10154000CDCDCDCDCDCDCDCDBC006E696368742041
:10155000616E67657363686C6F7373656E00206D91
:101560006D0020696E6368003E57656C6368652096
:10157000416368736520617566204E756C6C202828
:10158000782C792C7A2C61293F20000057656C63F8
:1015900068652041636873656E2073696E642061BD
:1015A0006E67657363686C6F7373656E20287879F6
:0615B0007A2C6C293F00BB
:00000001FF
